:101FA6002A56455253494F4E3A20522D444153200A
:101FB60056332E30002020202020200D0A002A4DE6
:101FC6003A2053656C6674657374206F6B0D0A0056
:101FD6002A573A2053656C66746573742066616986
:101FE6006C65640D0A002A52454144590D0A0000E9
:101FF6000000002A01005202007903009E0400C27C
:102006000500E50601060701270801460901640ADD
:1020160001E90F02581403001E03742803C3320398
:05202600F93C04023E3C
:100C8D00906EE5EEF0A3EFF0A37401F0906EE7E047
:100C9D00FF6412602AEF75F003A424F5F582E434A5
:100CAD001FF583E493FC740193FDC3906EE6E09D04
:100CBD00906EE5E09C4008906EE7E004F080CDEF8B
:100CCD0075F003A424F5F582E4341FF583E493FE57
:100CDD00740193FF906EE5E0FCA3E0FDC3EF9DFF73
:100CED00EE9CFEE4FCFDC8ECC8C9EDC9CAEECACB4A
:100CFD00EFCBA3E075F003A424F4F582E4341FF5E3
:100D0D0083E493FFE4FE1204EDECC0E0EDC0E0EEF1
:100D1D00C0E0EFC0E0906EE7E075F003A424F2F5BB
:100D2D0082E4341FF583E493FE740193FFC3906E48
:100D3D00E6E09FFF906EE5E09EFEE4FCFDC8ECC88A
:100D4D00C9EDC9CAEECACBEFCB906EE7E075F003E3
:100D5D00A424F7F582E4341FF583E493FFE4FE1237
:100D6D0004EDD0E0FBD0E0FAD0E0F9D0E0F8EF2BC5
:100D7D00FFEE3AFEED39FDEC38FC906EE8120644BC
:100D8D007FE87E037D007C00906EE8E0F8A3E0F93B
:100D9D00A3E0FAA3E0FB1204EDC8ECC8C9EDC9CA83
:100DAD00EECACBEFCB906EE7E0FF75F003A424F213
:100DBD00F582E4341FF583E493FC740193FDEF7524
:100DCD00F003A424F5F582E4341FF583C374019375
:100DDD009DFFE4939CC313FEEF13FFE4FCFDEB2F8B
:100DED00FFEA3EFEED39FDEC38FCECC0E0EDC0E075
:100DFD00EEC0E0EFC0E0906EE7E0FF75F003A424D5
:100E0D00F2F582E4341FF583E493FC740193FDEF56
:100E1D0075F003A424F5F582E4341FF583C3740142
:100E2D00939DFFE4939CFEE4FCFDF8F9CAEECACB5A
:100E3D00EFCBD0E0FFD0E0FED0E0FDD0E0FC12051E
:020E4D00782209
:1020A700201175906F81E05407906EDEF0C39403A2
:1020B7004066E064076061D2117F01122FB1E4909E
:1020C7006EDEF07F017D127B031230A0301706E52C
:1020D7006860F980397F017D0E7B031230A03017CD
:1020E70006E56860F980277F017D0A7B021230A030
:1020F700301706E56860F98015906EDEE004F0E0C1
:10210700B403C07F0112307C7F0A122FB1227F02F5
:0921170012307C7F0A122FB12264
:10153B003012030215D8E56864036009E568640B93
:10154B00600302163DC3E54F78D496FFE54E18961F
:10155B00FE120C8DCBEFCBCAEECAEB4A7003FA7BB3
:10156B0001D201E4906EDEF0CEEACECFEBCF7C0061
:10157B007D0A120436906EDEE024DFF582E4346ED1
:10158B00F583EDF0CEEACECFEBCF7C007D0A1204D3
:10159B0036CAEECACBEFCB906EDEE004F0E0B405BA
:1015AB00C7906EDE7404F0906EDEE0FFF46015748D
:1015BB00DF2FF582E4346EF583E07008906EDEE089
:1015CB0014F080E3EF04906EE4F0D212227F1E122F
:1015DB002FB17F017D327B041230A03017043016FF
:1015EB00FA227F0A122FB1906EE4E014906EDEF0B7
:1015FB00906EDEE024DFF582E4346EF583E0700B51
:10160B007F017D0B7B041230A08016906EDEE024F0
:10161B00DFF582E4346EF583E0FF7D0B7B01123046
:10162B00A03017043016FA22906EDEE0FF14F0EFB4
:03163B0070BE225C
:101E8B00D2AF122E61122FD412000E122E941230DA
:101E9B00DA12304E120003122120122F38122EF4B8
:101EAB007BFF7A1F79A6122B617BFF7A1F79BB12FE
:101EBB0000C9123044122A5650107BFF7A1F79C486
:101ECB001200C97F0112307C800B7BFF7A1F79D601
:101EDB001200C9D211121DF7906F13E0FF1229E403
:101EEB00122CC6122730906F14E0FEA3E0FF1228CD
:101EFB00E77BFF7A1F79EC1200C9C212C2113016B0
:101F0B0003122DD612153B906F0AE060F11220A739
:031F1B0080EC2235
:03000B00022209C5
:10220900C0E0C0F0C083C082C0D075D008C28CAF16
:102219008CEFFEAD8AED255F78D6F6E55E3E18F6C1
:10222900F58C08E6F58AD28CD56309906F09E0F53B
:1022390063122551D5621B906F09E0F5620561E5CE
:102249006170020560E56145607007E568600375C6
:102259006805E5686404600F12174012248C121C8B
:102269009D122B951226D7D0D0D082D083D0F0D012
:02227900E03251
:1028E700E4FCFDFB7AC079A8F81204ED7BE07A2EB0
:1028F700790078001228A3C374129FF55FE49EF550
:102907005E906F09E0F563F562E4F560F561E589CE
:1029170054F04401F589758CFF758AFFC2B9D2A9B5
:03292700D28C222D
:0C2FF000906F09E0F562E4F560F56122E5
:10273000E5C520E3FB75C50775C50FE5C530E4FBAE
:10274000AFC6EF75F004A4FFAEF0E5C5C413135493
:10275000037C002FF53CEC3EF53BE4F53AE53A25E9
:10276000E024BFF8A63B08A63CE53C2527F527E575
:102770003B3526F526053AE53AB40AE1E4F5392277
:10174000C0D075D00830190302183CE5C520E3FB72
:10175000E4F5C575C508F543754401E543640870B3
:101760000302181BE5C530E4FB85C62885C53DE5A9
:10177000436407600EE5C520E3FBE54304F5C5447B
:1017800008F5C5E52875F004A4FFAEF0E53DC413E7
:101790001354037C002FF546EC3EF545E54325E068
:1017A0002429F8A64508A646906F08E055446060D5
:1017B000AF28122AF9AF3D122AF9E543B40608858D
:1017C00045418546428049E54364077043E5392534
:1017D000E024C0F8C3E52796F527E5261896F526F8
:1017E000E53925E024BFF8A64508A646E5462527A5
:1017F000F527E5453526F526FEAF277C007D0A1244
:1018000004368E248F250539E539B40A03E4F53909
:101810000543E54425E0F54402175B300F1EE4A2C2
:10182000C492E4A2C592E5A29692E6A29792E72519
:0F18300068C4F53EAF3E122AF9853E40D0D02263
:10227B00C0D075D008300F65906F13E0FD7C0090D7
:10228B006F1BE0FB24FFFFE434FFFE120422EF245C
:10229B0001FFE43EFEC3E51F9FF51FE51E9EF51EE5
:1022AB008B3FE53F6021E51EF583E51FF582E0C41A
:1022BB0054F02568C4F0906F13E0251FF51FE4352B
:1022CB001EF51E153F80DB906F13E024FFFFE434F7
:1022DB00FFFEC3E51F9FF51FE51E9EF51ED0D02206
:0D2FE300E4F576F577F578C219122A1D2263
:10248C00C0D075D008E5686057201954122F9E40B3
:10249C004F906F13E02404906ED8F0906ED8E060EB
:1024AC003F20133C122B2D8F7512002E0577E577EC
:1024BC00700205767004E5766480701CF576F5770D
:1024CC000578E578B40C04D2198015122F8BE578B9
:1024DC0020E005122A1D8008906ED8E014F080BB15
:0324EC00D0D0222B
:102CC600E4906FAEF0A3F0906FAA120650000000D9
:102CD6000074FF78D3F608F6E4906FB0F0F569F566
:082CE60068906FA974FFF02251
:102E4700C0D075D008756801AF68122EC4C2901241
:0A2E57002FE37F0212307CD0D0225E
:102F0C00C0D0C291E5612401906FA8F0E4356090C7
:062F1C006FA7F0D0D022E7
:102F2200C0D0C292E5612401906FA8F0E4356090B0
:062F32006FA7F0D0D022D1
:1012E900C0D075D008E4906ED8F020C604E044015F
:1012F900F020C707906ED8E04402F0906FA9E0FF94
:10130900906ED8E0FE6F603BEE7025906FB6E0FFFF
:101319006005123084802C906FB5E0FF640360048F
:10132900EFB40405123084801A7F0112307C8013D7
:10133900906ED8E030E0077F0112308480057F028B
:10134900123084906ED8E0906FA9F0300B1EA294F1
:10135900300C01B34016C21A122FF0906F06E0FE4E
:10136900A3E0FF122BC5122E4702142A20100302F4
:10137900142A906F05E0C4F8540FC868FF906F04F1
:10138900E0C454F048FEC3E54D9FFDE54C9EFCE5E5
:1013990042C4F8540FC868FFE541C454F048FED36D
:1013A900EF9DEE9C4016D21A906FAA1206500000CB
:1013B9000000E4906FAEF0122FF08065C21A906FB2
:1013C900AAE0F8A3E0F9A3E0FAA3E0FBE8C0E0E5AE
:1013D90042C4F8540FC868FFE541C454F048FEC33D
:1013E900EF954DFFEE954CFE3395E0FDFCD0E0F80E
:1013F900EB2FFFEA3EFEE93DFDE83CFC906FAA12A7
:101409000644906F1BE0FF906FAEE004F06F70111F
:10141900906F0EE0FEA3E0FF122BC5122E47122299
:041429007BD0D02282
:101D5600C0D075D008906FAAE0F8A3E0F9A3E0FA26
:101D6600A3E0FBE8C0E0E542C4F8540FC868FFE50D
:101D760041C454F048FEC3EF954DFFEE954CFE333B
:101D860095E0FDFCD0E0F8EB2FFFEA3EFEE93DFDD5
:101D9600E83CFC906FAA120644300E387F007E00A5
:101DA6007D007C00906FAAE0F8A3E0F9A3E0FAA317
:101DB600E0FBD312060A401C906F03E0FFD3E561F7
:101DC6009FE5609400400D122F0C756802AF6812F3
:101DD6002EC4801A300D17906F19E065617002E508
:101DE60060700B122F0C75680AAF68122EC4D0D023
:011DF60022CA
:10219600C0D075D008906FA7E0FEA3E0656170031C
:1021A600E5606E7002D291300E3C906F11E0FEA396
:1021B600E0FFC3E54F9FFFE54E9EFEC3E5259FE585
:1021C600249E5007E4906FAFF0801B906F2CE0FFC9
:1021D600906FAFE004F06F700D122F22756803AF99
:1021E60068122EC4801A300D17906F1AE065617060
:1021F60002E560700B122F2275680BAF68122EC4B1
:03220600D0D02213
:102DF400C0D075D008906FA7E0FEA3E065617003B2
:0C2E0400E5606E7004D291D292D0D02212
:101C9D00C0D075D008E5687003021D2BE4F564759E
:101CAD006701E56464086065E56425E0241CF58240
:101CBD00E4346FF583E0FEA3E08E65F566F4700302
:101CCD00E565F4603EE56955677015E5616566701B
:101CDD0004E56065657009E5674269AF641227CC5C
:101CED00E5695567601DE5662401FFE43565FEEF86
:101CFD0065617003EE6560700AE567F45269AF6463
:101D0D0012285C0564E56725E0F5678095C3E52538
:101D1D0078D496E52418965005A62408A625E568DE
:101D2D0014601614601814601A24F96011146013ED
:101D3D00240B70121212E9800D121D56800812210B
:091D4D00968003122DF4D0D0227F
:1029E400CBEFCBEBFD7C007E3A7F98120436CDEB27
:1029F400CD7C001204228E1A8F1B74002FF582EEF8
:102A04003434AF82F5188F197E347F008E1C8F1DED
:092A14008E1E8F1FD213C2142282
:102AF900C213051FE51FAC1E7002051E14F5828C5A
:102B090083EFF0E51F65197004E51E6518700675F9
:102B19001E34751F00E51F651D7004E51E651C70D8
:042B290002D214229E
:102B2D00C214051DE51DAE1C7002051C14F5828E28
:102B3D0083E0FFE51D65197004E51C6518700675C9
:102B4D001C34751D00E51F651D7004E51E651C70A8
:042B5D0002D213226B
:102BC500C3E51F9FF51DE51E9EF51CC3E51D94007D
:102BD500E51C9434400BD3E51D9519E51C9518406B
:0E2BE5000CE51B251DF51DE51A351CF51C22FF
:101A2E002573202562752025627520257520257564
:101A3E00202562752025627520256320256275207C
:101A4E0025632025632025630D0A00632069676ED8
:101A5E0020257520257520257520257520257520B6
:101A6E0025752025752025750D0A006320786D6972
:101A7E007420257520256275202562750D0A006378
:101A8E0020677073202562750D0A00696E64657893
:101A9E00006572617365006F6666006F6E002A5690
:101AAE00455253494F4E3A20522D444153205633FE
:101ABE002E300D0A0063210063207264617300638F
:101ACE002069676E006320786D697400632067700B
:101ADE007300633F00630063200067707320007221
:101AEE0065736574002A453A20756E6B6E6F776E5E
:071AFE0020636D640D0A0076
:08000300E4F57DC216C21522CE
:1008F900906EDEEBF0A3EAF0A3E9F0300B13300CB5
:1009090008906EFB7401F0800D906EFB7402F0800C
:1009190005E4906EFBF0906EDEE0FBA3E0FAA3E045
:10092900F91203BA643F60030209D1906EE1E0F95C
:10093900A3E0FAA3E0906F30C9F0A3EAF0A3E9F0CD
:10094900906F09E0906F33F0906F08E0906F34F08A
:10095900906F04E0FFA3E0906F35CFF0A3EFF09024
:100969006F11E0FFA3E0906F37CFF0A3EFF0906F26
:1009790019E0906F39F0906F1AE0906F3AF0300FEC
:10098900047F3180027F30906F3BEFF0906EFBE087
:10099900906F3CF03010047F3180027F30906F3DC2
:1009A900EFF0300E047F3180027F30906F3EEFF020
:1009B900300D047F3180027F30906F3FEFF07BFF75
:1009C9007A1A792E1200C922906EDEE0FBA3E0FAB2
:1009D900A3E0F91203BAFF122F4E500C906EDFE418
:1009E90075F0011204C180E0E4906EFAF0906EDEB9
:1009F900E0FBA3E0FAA3E0F912142D906EFAE025CA
:100A0900E024E4F582E4346EF583EEF0A3EFF09090
:100A19006EDEE0FBA3E475F0011204D7A9F0FA1227
:100A290003BAFF122F4E50E7906EFAE004F0E0B4DB
:100A39000BBB906EE5E0906F09F0906EE7E0906F68
:100A490008F0906EE8E0FFA3E0906F04CFF0A3EF09
:100A5900F0906EEAE0FFA3E0906F11CFF0A3EFF002
:100A6900906EEDE0906F19F0906EEFE0906F1AF0D4
:100A7900906EF0E0FEA3E0FFEE4F24FF920FA3E09B
:100A8900FEA3E0FFEE4F24FF920BEF64014E7003CB
:100A9900D38001C3920C906EF4E0FEA3E0FFEE4F09
:100AA90024FF9210A3E0FEA3E0FFEE4F24FF920E75
:0D0AB900A3E0FEA3E0FFEE4F24FF920D220C
:10163E00906EDEEBF0A3EAF0A3E9F01203BA643F7A
:10164E0060030216D57BFF7A1A7959906F1CE0FF62
:10165E00A3E0906F30CFF0A3EFF0906F1EE0FFA3EA
:10166E00E0906F32CFF0A3EFF0906F20E0FFA3E099
:10167E00906F34CFF0A3EFF0906F22E0FFA3E090D5
:10168E006F36CFF0A3EFF0906F24E0FFA3E0906FE2
:10169E0038CFF0A3EFF0906F26E0FFA3E0906F3A03
:1016AE00CFF0A3EFF0906F28E0FFA3E0906F3CCF58
:1016BE00F0A3EFF0906F2AE0FFA3E0906F3ECFF023
:1016CE00A3EFF01200C922906EDEE0FBA3E0FAA3B6
:1016DE00E0F91203BAFF122F4E500C906EDFE47534
:1016EE00F0011204C180E0E4906EE1F0906EDEE055
:1016FE00FBA3E0FAA3E0F912142D906EE1E025E0D1
:10170E00241CF582E4346FF583EEF0A3EFF0906EB7
:10171E00DEE0FBA3E475F0011204D7A9F0FA120380
:10172E00BAFF122F4E50E7906EE1E004F0E0B408DD
:02173E00BB22CC
:101BD900906EDEEBF0A3EAF0A3E9F01203BAB43F8A
:101BE900297BFF7A1A7979906F0BE0FFA3E0906F58
:101BF90030CFF0A3EFF0906F18E0906F32F0906F54
:101C09000DE0906F33F01200C922906EDEE0FBA365
:101C1900E0FAA3E0F91203BAFF122F4E500C906EAE
:101C2900DFE475F0011204C180E0E4906EE7F09002
:101C39006EDEE0FBA3E0FAA3E0F912142D906EE743
:101C4900E025E024E1F582E4346EF583EEF0A3EFBC
:101C5900F0906EDEE0FBA3E475F0011204D7A9F061
:101C6900FA1203BAFF122F4E50E7906EE7E004F024
:101C7900E0B403BB906EE1E0FFA3E0906F0BCFF0FF
:101C8900A3EFF0906EE4E0906F18F0906EE6E090AC
:041C99006F0DF022B9
:1024EF00906EDEEBF0A3EAF0A3E9F0906EDEE0FB76
:1024FF00A3E0FAA3E0F91203BAB43F127BFF7A1AF2
:10250F00798D906F0AE0906F30F01200C922906EB3
:10251F00DEE0FBA3E0FAA3E0F91203BAFF122F4E9D
:10252F00500C906EDFE475F0011204C180E0906EE4
:10253F00DEE0FBA3E0FAA3E0F912142D906F0AEF8F
:02254F00F02278
:1006F9007B017A6E799A7D20122E10906EE1EBF0D3
:10070900A3EAF0A3E9F04A70047F0180027F009018
:100719006EEEEFF0605F7B017A6E799912142DC845
:10072900ECC8C9EDC9CAEECACBEFCB906F16E0FE93
:10073900A3E0FFE4FCFD1204EDC8ECC8C9EDC9CA89
:10074900EECACBEFCB906F06E0FEA3E0FFE4FCFD21
:10075900EB2FFFEA3EFEED39FDEC38FC906EE4121A
:100769000644906F16E0FEA3E0FFE4FCFD906EE8FE
:1007790012064480767B017A6E799912142DC8ECA1
:10078900C8C9EDC9CAEECACBEFCB906F13E0FFE43D
:10079900FCFDFE1204EDC8ECC8C9EDC9CAEECACB0E
:1007A900EFCB906F06E0FEA3E0FFE4FCFDEB2FFF2B
:1007B900EA3EFEED39FDEC38FC906EE412064490F9
:1007C9006EE1E0FBA3E0FAA3E0F912142DC8ECC82E
:1007D900C9EDC9CAEECACBEFCB906F13E0FFE4FCB9
:1007E900FDFE1204ED906EE8120644906EE4E0FC02
:1007F900A3E0FDA3E0FEA3E0FF780F1206318F7896
:10080900906EE4E0FCA3E0FDA3E0FEA3E0FFEE545C
:100819007FFEE48E768F77122F8B906EEEE0600963
:10082900E4906EECF0A3F0800B120026906EECEED3
:10083900F0A3EFF0E4906EDEF0A3F0906EDEE0FE40
:10084900A3E0FFE4FCFD906EE8E0F8A3E0F9A3E083
:10085900FAA3E0FBC3120620606C122FFC906EE035
:10086900EFF0906EEEE06014906EE0E0FF906EEDB8
:10087900E02FF0906EECE03400F08018906EECE020
:10088900FEA3E0FF906EE0E0FD12202B906EECEEEF
:10089900F0A3EFF0906EE0E0FF12306C0577E5779A
:1008A900700205767004E57664807009F576F5774F
:1008B9000578122F8B906EDFE004F07006906EDEE3
:1008C900E004F0020844906EEEE07013906EECE0E4
:1008D900FEA3E0FF123093906EECEEF0A3EFF090E0
:1008E9006EECE0FF12306C906EEDE0FF12306C227E
:102F6300D3EF648094B95007EF24D0FEFF8004EFC1
:042F730024A9FF226C
:10183F00906EDEEBF0A3EAF0A3E9F0906EE574FF93
:10184F00F0A3741AF0A37499F0A3E4F0A37405F055
:10185F001223C1EF7003122814906EE574FFF0A3EA
:10186F00741AF0A3749FF0A3E4F0A37405F0906EC4
:10187F00DEE0FBA3E0FAA3E0F91223C1EF7004123C
:10188F002E7B22906EE574FFF0A3741AF0A374A55B
:10189F00F0A3E4F0A37403F0906EDEE0FBA3E0FA94
:1018AF00A3E0F91223C1EF7003C21522906EE57405
:1018BF00FFF0A3741AF0A374A9F0A3E4F0A37402C9
:1018CF00F0906EDEE0FBA3E0FAA3E0F91223C1EF84
:1018DF007003D21522906EDEE0FBA3E0FAA3E0F9CD
:1018EF001203BAFF122C9D5043906EDEE0FBA3E073
:1018FF00FAA3E0F99000011203D3FF122F63CDEF8B
:10190F00CD906EDEE0FBA3E0FAA3E0F91203BAFF7D
:10191F00122F63EFC454F02DFF906EE1F0122EAC36
:0D192F00906EDFE475F0021204C180A92261
:0430CA00122D34226D
:0A3044007BFF7A1A79AC1200C92252
:100AC600906EE574FFF0A3741AF0A374C3F0A3E468
:100AD600F0A37402F07B017A6E79981223C1EF704D
:100AE60004120E4F22906EE574FFF0A3741AF0A361
:100AF60074C6F0A3E4F0A37406F07B017A6E7998CD
:100B06001223C1EF7018906EE174FFF0A3741AF00F
:100B1600A374C6F07B017A6E799E1208F922906E54
:100B2600E574FFF0A3741AF0A374CDF0A3E4F0A368
:100B36007405F07B017A6E79981223C1EF700A7BF7
:100B4600017A6E799D12163E22906EE574FFF0A32F
:100B5600741AF0A374D3F0A3E4F0A37406F07B0137
:100B66007A6E79981223C1EF700A7B017A6E799EAC
:100B7600121BD922906EE574FFF0A3741AF0A374C9
:100B8600DAF0A3E4F0A37405F07B017A6E7998128B
:100B960023C1EF700A7B017A6E799D1224EF2290B1
:100BA6006EE574FFF0A3741AF0A374E0F0A3E4F00A
:100BB600A37402F07B017A6E79981223C1EF701844
:100BC600906EE174FFF0A3741AF0A374E3F07B0156
:100BD6007A6E79991208F922906EE574FFF0A37483
:100BE6001AF0A374E5F0A3E4F0A37402F07B017A93
:100BF6006E79981223C1EF7018906EE174FFF0A31E
:100C0600741AF0A374E3F07B017A6E79991208F9ED
:100C160022906E98E0B464041206F922906EE57490
:100C2600FFF0A3741AF0A374E8F0A3E4F0A374042D
:100C3600F07B017A6E79981223C1EF700A7B017AF4
:100C46006E799C12183F22906EE574FFF0A3741A19
:100C5600F0A374EDF0A3E4F0A37405F07B017A6EC3
:100C660079981223C1EF70041230CA22906E98E070
:100C7600B4760412304422906E98E060097BFF7AC5
:070C86001A79F31200C922E4
:102DD60010160280107568047F0112307C7F1E1267
:0E2DE6002FB1120AC63015E81225B380E32281
:102A8F00C0D0EF20E72CEF640A6027EF640D6011D0
:102A9F007498257DF582E4346EF583EFF0057D8023
:102AAF00117498257DF582E4346EF583E4F0D21627
:052ABF00F57DD0D022DE
:102357002A4D4553534147453A2053746F72696E6E
:102367006720706172616D657465727320696E2094
:10237700464C4153480D0A002A4D455353414745A2
:102387003A2046696E69736865642073746F726971
:102397006E670D0A00000001C001C802000C001B97
:1023A7000100193C03FFFFFFFFFFFFFFFFFFFFFFD8
:0A23B700FFFFFFFFFF00000003001E
:0A304E00757923757A9C12117B221C
:10117B0090239CE49324FF920BA3E49324FF920C03
:10118B00A3E49324FF9210A3E493906F08F09023B1
:10119B00A0E49324FF920FE4906F13F07F80EF6035
:1011AB0014906F08E05F6007906F13E02402F0EF7C
:1011BB00C313FF80E9300F06906F13E004F0902308
:1011CB00A1E493906F09F09023A2E493906F10F039
:1011DB009023A3E493FF740193906F04CFF0A3EFDC
:1011EB00F09023A5E493FF740193906F11CFF0A3BC
:1011FB00EFF0906F09E0FBFD7C007E037FE81204AB
:10120B0036906F14EEF0A3EFF0906F13E0FA8BF0C3
:10121B00A4FF906F16E5F0F0A3EFF0EB1313543F20
:10122B00906F1BF0FB906F2CF09023A7E49324FF9F
:10123B00920EA3E49324FF920DA3E493906F19F005
:10124B009023AAE493906F1AF09023ABE493906FE2
:10125B0003F0906F10E0FF7E00906F16E0FCA3E0B0
:10126B00FD120422906F06EEF0A3EFF0EBFF7E0071
:10127B00EAFD7C00120422E02F906F0FF0906F06B6
:10128B00E03E906F0EF0E4FFEF25E024ACF582E436
:10129B003423F583E493FC740193FDEF25E0241CC8
:1012AB00F582E4346FF583ECF0A3EDF00FEFB408A7
:1012BB00D79023BCE493FF740193906F0BCFF0A3F3
:1012CB00EFF09023BEE493906F18F09023BFE4935C
:0E12DB00906F0DF09023C0E493906F0AF02204
:100E4F00A20BE433857A82857983F0A20CE433A375
:100E5F00F0A210E433857A82857983A3A3F0906F93
:100E6F0008E0857A82857983A3A3A3F0A20FE433E8
:100E7F00FFE57A2404F582E43579F583EFF0906F7E
:100E8F0009E0FFE57A2405F582E43579F583EFF083
:100E9F00906F10E0FFE57A2406F582E43579F5834B
:100EAF00EFF0906F04E0FEA3E0FFE57A2407F582F0
:100EBF00E43579F583EEF0A3EFF0906F11E0FEA328
:100ECF00E0FFE57A2409F582E43579F583EEF0A3A6
:100EDF00EFF0A20EE433FFE57A240BF582E43579C7
:100EEF00F583EFF0A20DE433FFE57A240CF582E4ED
:100EFF003579F583EFF0906F19E0FFE57A240DF562
:100F0F0082E43579F583EFF0906F1AE0FFE57A24EC
:100F1F000EF582E43579F583EFF0906F03E0FFE58E
:100F2F007A240FF582E43579F583EFF0E4906EDEE5
:100F3F00F0906EDEE0FF6408603BEF25E0241CF5C7
:100F4F0082E4346FF583E0FEA3E0FFE57A2410F529
:100F5F0082E43579F583C083C082906EDEE0D08263
:100F6F00D08375F002120681EEF0A3EFF0906EDEE3
:100F7F00E004F080BC906F0BE0FEA3E0FFE57A2465
:100F8F0020F582E43579F583EEF0A3EFF0906F183A
:100F9F00E0FFE57A2422F582E43579F583EFF090CE
:100FAF006F0DE0FFE57A2423F582E43579F583EFC1
:100FBF00F0906F0AE0FFE57A2424F582E43579F5A5
:100FCF0083EFF07BFF7A2379571200C9122AC47B73
:090FDF00FF7A23797F1200C92278
:101DF700E5C520E3FB75C50675C50EE5C530E4FBF3
:101E0700AFC6EF75F004A4FFAEF0E5C5C4131354D5
:101E1700037C002FF54DEC3EF54CE5C520E3FB7543
:101E2700C50775C50FE5C530E4FBAFC6EF75F00410
:101E3700A4FFAEF0E5C5C4131354037C002FF54A85
:101E4700EC3EF549F54E854A4FD21AE4F547F54879
:101E5700FFEF25E02455F582E4346FF583E54CF078
:101E6700A3E54DF0E54D2548F548E54C3547F547E1
:101E77000FEFB410DCE4F54BE5482410F54DE435DD
:041E870047F54C22AD
:10255100301A5EE5482410F54DE43547F54CE54B5E
:1025610025E02455F582E4346FF583E0FEA3E0FF16
:10257100C3E5489FF548E5479EF547E54B25E0242F
:1025810055F582E4346FF583E541F0A3E542F0E5CA
:10259100422548F548E5413547F547054BE54BB43C
:1025A1001003E4F54B85494E854A4F85244985251D
:0225B1004A22BC
:102E6100C21B43878075985AE589540F4420F58920
:0A2E7100758DFFD28ED2BCD2AC22C8
:03002300022C4B61
:102C4B00C0E0C0F0C083C082C0D075D010309807F0
:102C5B00AF99C298122A8F309904C299D21BD0D047
:092C6B00D082D083D0F0D0E03219
:08306C008F99301BFDC21B22ED
:083074008F99301BFDC21B22E5
:102C7400E5C520E3FB8FC5EF4408F5C5E5C530E4A1
:102C8400FBAFC6EF75F004A4FFAEF0E5C5C41313A3
:092C94005403FDE5F0EF4DFF22B1
:102D3400E4F5A8F5E8F5B8F5F875780FE578A2E0BC
:102D440092B5A2E192B3A2E292B4A2E392B202FFDC
:022D5400FE225D
:102F8B00E578A2E092B5A2E192B3A2E292B4A2E3F9
:032F9B0092B222CD
:0C2FFC00E5764480857782F583E0FF22B3
:10002E0090D3557499F090ACAA7466F090D3557431
:10003E0090F0E575F5F0E576D2E7F583E577F58294
:0D004E00E5F0F0E0A2E730F701B340F72243
:102A1D00E578A2E092B5A2E192B3A2E292B4A2E36C
:102A2D0092B290D3557499F090ACAA7466F090D38D
:102A3D00557480F090D3557499F090ACAA7466F0EB
:092A4D009080007414F0D21C22E8
:102F9E00301C0D908000E020E703D38001C3921C0B
:032FAE00A21C2240
:102AC40075780C122A1D122F9E40FB75780D122F5B
:102AD4008BE4F576F577857782857683E0F5751254
:102AE400002E0577E57770020576E5777004E576C4
:052AF400648070E22285
:0330DA00C21C22F3
:03005B000222EB93
:1022EB00C0E0C0D0C2CC742D25C9F5C93017581524
:1022FB0050E5507052E55670128552FCC2C0F55134
:10230B00755601E55425E0F550803CE556640170A7
:10231B002375FCFFD2C00551E5516553700E301883
:10232B0007F556855550801FC217801B75560275D1
:10233B0050028013E556B4020E8552FCC2C075568E
:0C234B0001E55425E0F550D0D0D0E03280
:102E940075FCFFD2C075FE0B75528075EA0DC2FC3D
:082EA400D2EC75550AC2172299
:102CEE00C217A202921875FCFFD2C08F53E4F5569C
:102CFE00CEEDCE8EFECEEBCE8E54855550EF6002CD
:032D0E00D21722B7
:06309A00D202122CEE220E
:0630A000C202122CEE2218
:08307C007D0B7B0112309A224A
:083084007D327B0412309A2218
:102FB100C21775FCFFD2C08F55E4F556855550D226
:022FC1001722D5
:101B05002A4D3A20615F7374203D2025750D0A002A
:101B15002A4D3A2061283029203D2025750D0A00DF
:101B25002A573A20615F73743D25752C2061303D3D
:101B350025752028672D73772064697361626C654C
:101B450064290D0A002A4D3A2070283029203D20AD
:101B550025750D0A002A573A20502072616E676577
:101B6500205B25752C25755D0D0A002A573A204204
:101B750057206572726F722028425720646973611D
:101B8500626C6564290D0A002A573A206E6F206938
:101B9500676E202562640D0A002A573A206E6F2071
:101BA500786D69740D0A002A573A206E6F206770A8
:101BB500730D0A002A573A2064726F6775652065B0
:101BC50072720D0A002A573A206D61696E2065729E
:041BD500720D0A0083
:07308C00EF60031F80FA2230
:102DB700A2029293E4F57BF57C7F7812308C057C38
:0F2DC700E57C7002057BE57C640A457B70EB229E
:100FE800E4906EE3F0906EDEF0A3F0906EE2F0D243
:100FF80002122DB77F06122C74906EDFE02FF0904E
:101008006EDEE03EF0C202122DB7906EE2E004F010
:10101800E0B420DB906EDEE0FEA3E0FF7C007D20E4
:1010280012048B906EDEEEF0A3EFF07BFF7A1B7953
:1010380005906F30EEF0A3EFF01200C9E4906EE077
:10104800F0A3F0A3F07F06122C74906EE1E02FF06D
:10105800906EE0E03EF0906EE2E004F0E0B420E54F
:10106800906EE0E0FEA3E0FF7C007D2012048B90F0
:101078006EE0EEF0A3EFF07BFF7A1B7915906F30EE
:10108800EEF0A3EFF01200C9906EE0E0FEA3E0FFDF
:10109800906EDEE0FCA3E0FDC39FFFEC9EFEC3EF75
:1010A800942DEE64809480502D7BFF7A1B792590D7
:1010B8006F30ECF0A3EDF0906EE0E0FFA3E0906FEE
:1010C80032CFF0A3EFF01200C97F06123084C210AD
:1010D800906EE37406F0E4906EDEF0A3F0906EE29A
:1010E800F07F07122C74906EDFE02FF0906EDEE038
:1010F8003EF0906EE2E004F0E0B420E5906EDEE0B1
:10110800FEA3E0FF7C007D2012048B906EDEEEF0E3
:10111800A3EFF07BFF7A1B794A906F30EEF0A3EFD4
:10112800F01200C9906EDEE0FEA3E0FFC3947DEEEE
:1011380064809482400BD3EF94DBEE648094834008
:101148002C7BFF7A1B795A906F30EEF0A3EFF0A357
:101158007402F0A3747DF0A37403F0A374DBF0129F
:1011680000C97F05123084906EE37405F0906EE339
:03117800E0FF2273
:10193C00E4906EDEF0300B1EA294300C01B3401616
:10194C007BFF7A1B79701200C97F03123084C20BA3
:10195C00906EDE7403F0E4906EDFF0906EDFE0FFCB
:10196C006408606AEF25E0241CF582E4346FF5838B
:10197C00E0FCA3E0F47002ECF4604B123008401F62
:10198C007F041230847BFF7A1B798D906EDFE0042C
:10199C00906F30F01200C9906EDE7404F0802790C6
:1019AC006EDFE0FF122780401D7F041230847BFF26
:1019BC007A1B798D906EDFE004906F30F01200C9C5
:1019CC00906EDE7404F0906EDFE004F0808D906F0A
:1019DC000BE07002A3E060201230AC401B7F0412BD
:1019EC0030847BFF7A1B799E1200C9E4906F0BF058
:1019FC00A3F0906EDE7404F0906F0AE0601E12305B
:101A0C00A640197F041230847BFF7A1B79AC12003C
:101A1C00C9E4906F0AF0906EDE7404F0906EDEE014
:021A2C00FF2297
:102A5600D20112193C906FB5EFF06002C201120F5D
:102A6600E8906FB6EFF06002C20120C60B7BFF7ADA
:102A76001B79B91200C9C20120C70B7BFF7A1B79EB
:092A8600CA1200C9C201A201221A
:10000E00E4FF74B12FF582E4346FF58374FFF00FC3
:05001E00EFB404EE2226
:0C300800EFC31325E02441FF122E2C2200
:10278000906EE0EFF0E0FFC31325E02441FF7B01F2
:102790007A6E79E2906EE87401F012292A906EE167
:1027A000EFF0906EE0E054012402FF74017E00C857
:1027B000EFC8088005C333CE33CED8F9FF906EE260
:0C27C000E0FDE4EF5D6003D38001C32264
:1027CC00CEEFCEEEC313FF24B1F582E4346FF58364
:1027DC00C083C082E0FDEE5401FC7401C8ECC80853
:1027EC008002C333D8FCF45DD082D083F0EF25E0B7
:1027FC002440FFEEC31324B1F582E4346FAD82FCA8
:08280C007B01D2011229A9226F
:10285C00CEEFCEEEC313FF24B1F582E4346FF583D3
:10286C00C083C082E0FDEE5401FC7401C8ECC808C2
:10287C008002C333D8FC4DD082D083F0EF25E02406
:10288C0040FFEEC31324B1F582E4346FAD82FC7BC0
:07289C0001D2011229A9225B
:102F3800E4F57EFF74752FF582E4346FF583E4F0D1
:062F48000FEFB40DEF22B3
:0630A6007F50122E2C22C7
:102EAC00906EE2EFF07F507C6E7DE27B01D20112DE
:082EBC0029A9906EE3EFF0225A
:1025B3007F537B017A6E79DF906EE87401F0122904
:1025C3002A906EDEEFF0A3E0D3941040037410F072
:1025D300906EDFE0FE603A7F517B017A6F798290E3
:1025E3006EE8F012292A906EDEEFF0E4F0906EDFD1
:1025F300E0FF906EDEE0FE6F601774822EF582E4DA
:10260300346FF583E0FF123074906EDEE004F080E7
:02261300DC22C7
:10281400E4906EE2F07F577B017A6F7982906EE8E4
:102824007410F012292A906EE3EFF0E4F0906EE356
:10283400E0FF6410601774822FF582E4346FF5832F
:10284400E0FF123074906EE3E004F080E0906EE2FA
:08285400E004F0E0B408BE222C
:102E7B00906EE27442F07F567C6E7DE27B01D20154
:092E8B001229A9906EE3EFF02278
:102EC400906ED9EFF07F547C6E7DD97B01C20112E4
:082ED40029A9906EDAEFF0224B
:102B9500C0D075D008906F0AE06022057E906F095D
:102BA500E0657E7018F57E7F557B017A6F797590AB
:102BB5006EE8740DF012292A906ED8EFF0D0D0226D
:10212000E4F557F558F559906F09E0FF75F00A840A
:10213000755C00F55DEFC313755A00F55B906F0B8E
:10214000E0FEA3E0FF4E604D906F927404F0E4A3B4
:10215000F0FCFDF8F9CAEECACBEFCBFF7EC07DA83C
:102160001228A37B107A00790078001228A3EF14BC
:10217000906F94F0906F0DE0FF33333354F8FF907D
:102180006F18E02F906F95F07F607C6F7D927B04DD
:06219000D2011229A92270
:0630AC007F60122E2C22B1
:10242800906F927415F0A37401F0E558A3F0E55984
:10243800A3F0E529A3F0E52AA3F0E52BA3F0E52C0A
:10244800A3F0E52DA3F0E52EA3F0E52FA3F0E530EA
:10245800A3F0E531A3F0E532A3F0E533A3F0E534CA
:10246800A3F0E535A3F0E536A3F0E537A3F0E538AA
:10247800A3F0A3E540F07F607C6F7D927B15C201DD
:042488001229A9224A
:101F1E00906F927415F0A37402F0E558A3F0E55992
:101F2E00A3F0906F75E0906F96F0906F76E0906FE3
:101F3E0097F0906F77E0906F98F0906F78E0906FD9
:101F4E0099F0906F79E0906F9AF0906F7AE0906FC1
:101F5E009BF0906F7BE0906F9CF0906F7CE0906FA9
:101F6E009DF0906F7DE0906F9EF0906F7EE0906F91
:101F7E009FF0906F7FE0906FA0F0906F80E0906F79
:101F8E00A1F0906F81E0906FA2F07F607C6F7D92E8
:081F9E007B11C2011229A922E6
:1026D700C0D075D008906F0BE07002A3E06047058B
:1026E70057906F09E065577002F557AF577E00ACFA
:1026F7005CAD5D120436ED4C700F122428E568605E
:10270700080559E55970020558AF577E00AC5AAD18
:102717005B120436E55CC313FEE55D136D7002ECD6
:092727006E7003121F1ED0D022B7
:102D77000000CC01D8011400F0013C002800E40158
:102D8700A0016C007800B40150009C018801440048
:050026007EFF7FFF22B8
:10202B00CBEFCBCAEECAC9EDC9E9540FFFEAEB6F90
:10203B00540F25E0FFE433FE74772FF582EE342D39
:10204B00F583EAC4F854F0C868FEEBC4540F48FF9C
:10205B00EE540FFEE4936EFA7401936FFBCFE9CF4E
:10206B00EFC4540F540FFFEAEF6B540F25E0FFE45E
:10207B0033FE74772FF582EE342DF583EAC4F854D2
:10208B00F0C868FEEBC4540F48FFEE540FFEE49308
:0C209B006EFA7401936FFBCEEACEFF22B8
:07309300EEF4FEEFF4FF2252
:10267700FF30CEFF3058FF3062FF2D56FF30B2FFDC
:102687002D11FF30B8FF30D2FF2EDCFF30BEFF2DFB
:1026970097FF2F77FF30D6FF30DDFF30DEFF30DFCB
:1026A700FF30E0FF30E1FF30E2FF30E3FF30E4FFCF
:1026B70030E5FF30E6FF30E7FF30E8FF30E9FF3075
:1026C700C4FF30C4FF30C4FF30C4FF30C4FF30C480
:0F2FD400D296D29775D8C575DBECD2BDD2AD229F
:102E2C00E4F56F8F6DD21DD2DDFF122C20EF6418EC
:0B2E3C006004EFB44003D38001C32208
:1029A900906EE5ECF0A3EDF08C838D82787FEBFEE1
:1029B9006006E0F6A308DEFA8B6F8F6DD21DD2DDBB
:1029C90030010DCFEBCF122C20906EE7EFF0800590
:0B29D900E4906EE7F0906EE7E0FF2254
:10292A00906EE5EBF0A3EAF0A3E9F0CEEFCEA3E0D8
:10293A00FFF56F8E6DD21DD2DD122C20E4FE906E53
:10294A00E8E06E601D747F2EF8E6FD906EE5E0FB10
:10295A00A3E0FAA3E0F98E82758300ED1204000E5B
:03296A0080DC22EC
:102C2000CEEFCEE4F56AEE2402FDE433FCE56A6DF6
:102C30007001EC6010756BDDD56BFD201D03AF6E70
:0B2C400022056A80E175D8D57F0022D4
:0430CE0075D8D522BA
:0A305800856DDA75D8C5E4F56C2229
:0A306200856DDA75D8C5E4F56C221F
:102D5600C0D075D010E56F700775D8D5C21D800E2E
:102D6600AF6C056C747F2FF8E6F5DA75D8C5D0D050
:012D7600223A
:0630B20075D8D5C21D22F5
:102D1100C0D075D010E56C656F700775D8D5C21D30
:102D2100800EAF6C056C747F2FF8E6F5DA75D8C5A7
:032D3100D0D022DD
:0630B80075D8D5C21D22EF
:0430D20075D8E522A6
:102EDC00E56F14600A04700C75D8D5C21D80087596
:082EEC00D8C1800375D8C5228E
:0630BE0075D8D5C21D22E9
:102D9700C0D075D010747F256CF8A6DAE56F1405DE
:102DA7006C656C700575D8C1800375D8C5D0D02205
:102F7700C0D075D010747F256CF8A6DA75D8D5C285
:042F87001DD0D02267
:0430D60075D8D522B2
:0130DD0022D0
:0130DE0022CF
:0130DF0022CE
:0130E00022CD
:0130E10022CC
:0130E20022CB
:0130E30022CA
:0130E40022C9
:0130E50022C8
:0130E60022C7
:0130E70022C6
:0130E80022C5
:0130E90022C4
:0630C40075D8D5C21D22E3
:03002B0002296D3A
:10296D00C0E0C0F0C083C082C0D075D01085D96ED4
:10297D00E5D9131313541F75F003A42477F582E4DE
:10298D003426F583E493740193FA740293F91206D5
:0C299D008DD0D0D082D083D0F0D0E032BA
:0C301400122615EF3395E0EF20E7F522BF
:102BF300ED7804A2E713D8FB2FFE2440906EE1F09A
:102C0300A3EEF0ED540F2FFE2440A3F0A3EEF07FCC
:0D2C1300487C6E7DE17B04D2011229A922CC
:102EF4007F281230207F011230201230147F0C12F0
:082F040030207F021230202270
:0C302000CEEFCEE4FFCDEECD122BF3225C
:0C302C00CEEFCE7F20CDEECD122BF32294
:102B6100906EDEEBF0A3EAF0A3E9F0906EDEE0FBFD
:102B7100A3E0FAA3E0F91203BA6018906EDEE0A3B5
:102B8100E475F0011204D7A9F0FA1203BAFF12306A
:042B91002C80D8229A
:10261500906EDE7450F0A37410F07F487C6E7DDE02
:102625007B02D2011229A97F497B017A6E79E0905C
:102635006EE87401F012292A906EDE7450F0A374CE
:1026450010F07F487C6E7DDE7B02D2011229A97FC6
:10265500497B017A6E79E1906EE87401F012292ABE
:10266500906EE0E0540FFFC454F0FFA3E0540F2F29
:02267500FF2242
:0300000002303893
:0C303800787FE4F6D8FD7581D6021E8B6F
:1003BA00BB010689828A83E0225002E722BBFE0241
:0903CA00E32289828A83E4932274
:1003D300BB010CE58229F582E5833AF583E02250DF
:1003E30006E92582F8E622BBFE06E92582F8E22229
:0D03F300E58229F582E5833AF583E4932243
:10040000F8BB010DE58229F582E5833AF583E8F032
:10041000225006E92582C8F622BBFE05E92582C8DE
:02042000F222C6
:10042200EFF88DF0A4FFEDC5F0CEA42EFEEC88F01F
:04043200A42EFE22D4
:10043600BC000BBE0029EF8DF084FFADF022E4CCAA
:10044600F875F008EF2FFFEE33FEEC33FCEE9DEC73
:10045600984005FCEE9DFE0FD5F0E9E4CEFD22EDB9
:10046600F8F5F0EE8420D21CFEADF075F008EF2F03
:10047600FFED33FD4007985006D5F0F222C398FDF4
:050486000FD5F0EA2291
:10048B00C2D5EC30E709B2D5E4C39DFDE49CFCEE8C
:10049B0030E715B2D5E4C39FFFE49EFE120436C3CA
:1004AB00E49DFDE49CFC800312043630D507C3E4C5
:0604BB009FFFE49EFE22FB
:1004C100C5F0F8A3E028F0C5F0F8E58215827002C6
:0604D1001583E038F02263
:1004D700A3F8E0C5F025F0F0E582158270021583D8
:0604E700E0C838F0E82235
:1004ED00E88FF0A4CC8BF0A42CFCE98EF0A42CFCAE
:1004FD008AF0EDA42CFCEA8EF0A4CDA8F08BF0A42C
:10050D002DCC3825F0FDE98FF0A42CCD35F0FCEB8A
:10051D008EF0A4FEA9F0EB8FF0A4CFC5F02ECD394F
:0F052D00FEE43CFCEAA42DCE35F0FDE43CFC22BC
:10053C0075F008758200EF2FFFEE33FECD33CDCC76
:10054C0033CCC58233C5829BED9AEC99E5829840F9
:10055C000CF582EE9BFEED9AFDEC99FC0FD5F0D6D6
:10056C00E4CEFBE4CDFAE4CCF9A88222B800C1B900
:10057C000059BA002DEC8BF084CFCECDFCE5F0CB3E
:10058C00F97818EF2FFFEE33FEED33FDEC33FCEB77
:10059C0033FB10D703994004EB99FB0FD8E5E4F932
:1005AC00FA227818EF2FFFEE33FEED33FDEC33FC1F
:1005BC00C933C910D7059BE99A4007EC9BFCE99A13
:1005CC00F90FD8E0E4C9FAE4CCFB2275F010EF2F58
:1005DC00FFEE33FEED33FDCC33CCC833C810D70758
:1005EC009BEC9AE899400AED9BFDEC9AFCE899F893
:0E05FC000FD5F0DAE4CDFBE4CCFAE4C8F92226
:1028A300C2D5E830E70FB2D5E4C39BFBE49AFAE460
:1028B30099F9E498F8EC30E717B2D51228D9120544
:1028C30078E4C39BFBE49AFAE499F9E498F880036B
:1028D30012057830D50DE4C39FFFE49EFEE49DFD11
:0428E300E49CFC2253
:10060A00EB9FF5F0EA9E42F0E99D42F0EC6480C867
:06061A0064809845F02207
:10062000EB9FF5F0EA9E42F0E99D42F0E89C45F030
:0106300022A7
:10063100E8600FECC313FCED13FDEE13FEEF13FFA7
:03064100D8F122CB
:0C064400ECF0A3EDF0A3EEF0A3EFF02229
:10065000A8828583F0D083D08212066712066712C3
:100660000667120667E473E493A3C583C5F0C583E8
:10067000C8C582C8F0A3C583C5F0C583C8C582C8F4
:010680002257
:0C068100A42582F582E5F03583F5832284
:06068D008A838982E473F8
:10005E00E5702430F582E4346FF583E0057022906C
:10006E006F2D300903906F30E475F0011206B30264
:10007E0003BA2002E97F2ED2028018EF540F24908B
:10008E00D43440D4FF30060BEF24BFB41A00500313
:10009E002461FFE571600215710574E57470020547
:1000AE007330090E906F2DE475F0011206B3EF0256
:1000BE0006930230747403D2098003E4C209F5700A
:1000CE00906F2D1206CAE4F571F573F574E5716043
:1000DE00077F201200A180F5F572C203C202C2048E
:1000EE00C205C207C208C20A12006DFF700D3009A8
:1000FE00057F001200B2AF74AE7322B42561C2D573
:10010E00C20612006DFF24D0B40A00501C75F00A0E
:10011E0020D50DC571A42571F5717002D20580E050
:10012E00C572A42572F57280D724CFB41A00EF5091
:10013E0004C2E5D2060202ACD20380C4D20280BE53
:10014E00D20480BAD2D580B8D20780B27F201200F6
:10015E00A12004077401B5710040F112005EFF1278
:10016E0000A10200DBD20AD208809312005EFB12BD
:10017E00005EFA12005EF94A4B700679787A037BBC
:10018E00FF200433E571602FAF72BF00011F7E00A8
:10019E008E827583001203D360050EEE6F70F1C26E
:1001AE00D5EBC0E0EAC0E0E9C0E0EE1202F0D0E02C
:1001BE00F9D0E0FAD0E0FB1203BAFF60A5EBC0E085
:1001CE00EAC0E0E9C0E01200A1D0E02401F9D0E0DD
:1001DE003400FAD0E0FBE57260DDD572DA80837B05
:1001EE00FF7A0279ECD2048098791080027908C2E5
:1001FE0008C20A8008D2D5790A8004790AC2D5E4E9
:10020E00FAFDFEFF12005EFC7B0820031312005E57
:10021E00FD7B1030020A12005EFE12005EFF7B2094
:10022E00EC3382D592D55013C3E43002069FFFE41F
:10023E009EFEE42003039DFDE49CFCE4CBF8C20388
:10024E00EC700CCFCECDCCE824F8F870F38017C349
:10025E00EF33FFEE33FEED33FDEC33FCEB33FB9966
:10026E004002FB0FD8E9EB300305F8D0E0C448B2EA
:10027E0003C0E00AEC4D4E4F78207B0070C2EAC0FE
:10028E00E01202F2D0F0D0E0200304C4C0E0C4B209
:10029E0003C0F012008AD0F0D5F0EB0200DB12069C
:1002AE00D301795301F758014A4C01464201FB4FE5
:1002BE00020344020349015F4302095501ED460161
:1002CE00ED4501ED47039B50014E2D01522E017558
:1002DE002B01562301732003862A0000016D3F3F38
:1002EE003F00790AA2D5200514300709B91002047F
:1002FE0004B9080104A2D5200802500104200466A6
:02030E00920457
:10031000B571005032C0E07F203005177F30A20455
:1003200072087207500D120347C204C208C2077F49
:1003300030800F300703E9C0E01200A1300703D07E
:10034000E0F9D0E0B571CE3007177F30B9100C124C
:1003500000A17F583006077F788003B90803120098
:10036000A13004057F2D0200A17F20200AF87F2BF9
:100370002008F322920480CF286E756C6C29002D22
:1003800050434958D20312005E3003F8C20378711B
:1003900030D504D2027872F602010C12005E2403FA
:1003A000B405004001E490037F93120092743A1266
:0A03B0000092D2057571040201F7F6
:102F4E00EFC394094006EFC3940E4004EFB4200380
:052F5E00D38001C32235
:102C9D00EFC394414006EFC394474018EFC39461CE
:102CAD004006EFC39467400CEFC394304009EFC367
:092CBD00943A5003D38001C322B4
:1023C100906EE2EBF0A3EAF0A3E9F0906EE5E0FB9A
:1023D100A3E0FAA3E0F91203BAFE906EE2E0FBA3D8
:1023E100E0FAA3E0F91203BAFD6E702AED600E90D7
:1023F1006EE874FFF5F01204C145F070037F00220E
:10240100906EE3E475F0011204C1906EE6E475F09C
:10241100011204C180B5D3EE6480F8ED6480984068
:07242100037F01227FFF226F
:102E1000E94A4B7001221203BAFF6D700122EF7074
:0C2E200004FBFAF92209E970ED0A80EACF
:10142D00906EFCEBF0A3EAF0A3E9F0906EFCE0FB0C
:10143D00A3E0FAA3E0F91203BAFF122F4E500C905D
:10144D006EFDE475F0011204C180E0D201906EFCD6
:10145D00E0FBA3E0FAA3E0F91203BAFF642B6004EA
:10146D00EFB42D1D906EFCE0FBA3E475F0011204AA
:10147D00D7A9F0FA1203BA642D6003D38001C39289
:10148D0001906EFF12065000000000906EFCE0FB14
:10149D00A3E0FAA3E0F91203BAFF122FC3506A7F3B
:1014AD000A7E007D007C00906EFFE0F8A3E0F9A3BA
:1014BD00E0FAA3E0FB1204EDC8ECC8EDC0E0EEC00D
:1014CD00E0EFC0E0906EFCE0FBA3E0FAA3E0F912C0
:1014DD0003BAFF3395E0FEEF24D0FFEE34FFFEE4B8
:1014ED00FCFDD0E0FBD0E0FAD0E0F9EB2FFFEA3EB7
:1014FD00FEED39FDEC38FC906EFF120644906EFD4A
:10150D00E475F0011204C18082300110906EFFE08D
:10151D00FCA3E0FDA3E0FEA3E0FF8011906EFFE0D1
:0E152D00FCA3E0FDA3E0FEA3E0FF1206A52252
:10069300BB010689828A83F0225002F722BBFE0146
:0206A300F32240
:0E06A500C3E49FFFE49EFEE49DFDE49CFC2266
:1006B300F8E0FBA3A3E0F925F0F0E58215827002D0
:0706C3001583E0FA38F02274
:0906CA00EBF0A3EAF0A3E9F02231
:1006D300D083D082F8E4937012740193700DA3A3B6
:1006E30093F8740193F5828883E4737402936860CA
:0606F300EFA3A3A380DFCA
:102FC300EFC394304009EFC3943A5003D38001C355
:012FD30022DB
:00000001FF
